:100000008A110A1205280000090007309F00831694
:100010008601850183125830C8000230C90037308C
:10002000C000C1014008C2004108C3004008A6004A
:100030004108A7000430A200A3014C25C4002508F4
:10004000C5004008A6004108A7000C30A200A3018B
:100050004C25C6002508C700F430A0000130A100DF
:10006000622586110512831686110512F03085056A
:1000700083126430A0000030A10062253330BF2518
:100080003330BF253330BF252230BF252830BF2570
:100090000D30BF250130BF250130BF258030BF2581
:1000A0002030A7254230A7256130A7256C30A72531
:1000B0006930A7257A30A7256130A7252030A725EC
:1000C0002030A7254C30A7255530A7253230A7254D
:1000D0004430A7254930A7254D30A7252030A72536
:1000E000C830A000A101622586172C30A000013085
:1000F000A1006225AF218613AE012E08023C031C2D
:10010000FA288122AC012C080F3C031C92282A30CB
:10011000B0001C250F30A000A10162250130AC0702
:10012000031C83281F308305F430A0000130A10098
:100130006225AC012C080F3C031CC2282C080F3C84
:10014000031CB928A520B000B92800308A002C086B
:1001500082072034203420342034203420342034CA
:1001600020342034203420342034203420342034EF
:1001700020341C250F30A000A10162250130AC07FE
:10018000031C9A281F308305D030A0000730A1003F
:1001900062250130BF252C30A0000130A10062256E
:1001A0008030BF252030A7254230A7256130A72504
:1001B0006C30A7256930A7257A30A7256130A7259F
:1001C0002030A7252030A7254C30A7255530A7255E
:1001D0003230A7254430A7254930A7254D30A72523
:1001E0002030A725C830A000A10162250130AE074C
:1001F000031C7D281F308305061681220612AE01DE
:100200002E08023C031C7D298122AC012C080F3CE6
:10021000031C15292A30B0001C250F30A000A101B5
:1002200062250130AC07031C06291F308305F4301A
:10023000A0000130A1006225AC012C080F3C031C7A
:1002400045292C080F3C031C3C292821B0003C29DF
:1002500001308A002C0882072034203420342034D6
:1002600020342034203420342034203420342034EE
:1002700020342034203420341C250F30A000A1016C
:1002800062250130AC07031C1D291F308305D030C7
:10029000A0000730A10062250130BF252C30A0004E
:1002A0000130A10062258030BF252030A7254230D3
:1002B000A7256130A7256C30A7256930A7257A309E
:1002C000A7256130A7252030A7252030A7254C3051
:1002D000A7255530A7253230A7254430A72549301A
:1002E000A7254D30A7252030A725C830A000A101A3
:1002F00062250130AE07031C00291F308305AF21A2
:100300000130BF252C30A0000130A10062258030D3
:10031000BF252030A7254230A7256130A7256C30A6
:10032000A7256930A7257A30A7256130A725203079
:10033000A7252030A7254C30A7255530A7253230DA
:10034000A7254430A7254930A7254D30A7252030C3
:10035000A725C830A000A10162257C28AE29061679
:100360002C30A0000130A1006225AC012C080F3C0C
:10037000031CC5292A30B0001C250A30A000A101A9
:1003800062250130AC07031CB6291F308305F43009
:10039000A0000130A1006225AC012C080F3C031C19
:1003A000F5292C080F3C031CEC29D821B000EC29BE
:1003B00001308A002C088207203420342034203475
:1003C000203420342034203420342034203420348D
:1003D00020342034203420341C251430A000A10106
:1003E00062250130AC07031CCD291F3083055F3027
:1003F000B0001C2531245630B0001C25B524312412
:100400005630B0001C25B52431245630B0001C25D0
:10041000C7245F30B0001C25AC012C08023C031C33
:10042000362A0A244C30B0001C25B5242D24553022
:10043000B0001C25B52455243230B0001C25B5244D
:10044000EA234430B0001C25B524FE234930B00017
:100450001C25B5240F244D30B0001C25C7245F3067
:10046000B0001C250130AC07031C0D2A1F3083058A
:10047000EA234430B0001C25B52419245030B000C4
:100480001C25C7245F30B0001C2555243230B00035
:100490001C25B52436245730B0001C25C7245F30F6
:1004A000B0001C25F5234730B0001C25B524F023EF
:1004B0004630B0001C25B52449243030B0001C253E
:1004C000B52467243530B0001C25B5241E245130D6
:1004D000B0001C25B52415244F30B0001C25C724BE
:1004E0005F30B0001C250925FF30B0001C255F30AF
:1004F000B0001C258122C830A000A101622506128F
:100500000800AC012C080F3C031C912A2A30B000D3
:100510001C253230A000A10162250130AC07031C6C
:10052000822A1F3083055830A0000230A1006225C6
:10053000AC012C080F3C031CC12A2C080F3C031CE7
:10054000B82AA422B000B82A02308A002C088207F8
:1005500020342034203420342034203420342034FB
:1005600020342034203420342034203420342034EB
:100570001C253230A000A10162250130AC07031C0C
:10058000992A1F3083055830A0000230A10062254F
:10059000AC012C08183C031CFB2A2C08183C031C3B
:1005A000F12AD422B000F12A02308A002C088207F6
:1005B0002034503472346F34793465346334743495
:1005C0006F342034203420342034503452344534B5
:1005D000533445344E344334493441342034203488
:1005E00020341C250E30A0000130A100622501300E
:1005F000AC07031CC92A1F308305BC30A0000230A1
:10060000A1006225AC012C080F3C031C2B2B2C08ED
:100610000F3C031C222B0E23B000222B03308A0038
:100620002C08820720342034203420342034203415
:10063000203420342034203420342034203420341A
:10064000203420341C253230A000A1016225013065
:10065000AC07031C032B1F308305AC012C08323C74
:10066000031C7A2B2C08323C031C702B3923B0005E
:10067000702B03308A002C088207523461346434B2
:1006800069346F34623461346C3469347A3461347F
:10069000203465346E3420346734753461347234F8
:1006A000643461342034643465346C3420344D3423
:1006B0007534733465346F3420344E346134763499
:1006C00061346C3420346434653420346C346134E7
:1006D00020344E346134633469346F346E342034E2
:1006E0001C250E30A0000130A10062250130AC07AE
:1006F000031C2E2B1F308305AC012C083E3C031C31
:10070000D52B2C083E3C031CCB2B8823B000CB2BD5
:1007100003308A002C0882076834613473347434DF
:1007200061342034733465347234203469346E3467
:100730007334743461346C3461346434613420341F
:1007400064346534663469346E34693474346934BD
:10075000763461346D3465346E34743465342034E9
:1007600065346E3420344E347534653473347434E7
:100770007234613473342034493453344C3441344A
:10078000533420344D3441344C34563449344E348F
:100790004134533420341C250E30A0000130A10018
:1007A00062250130AC07031C7D2B1F308305E83028
:1007B000A0000330A10062250800E324F62408000D
:1007C000F624E324E324E3240800F624E324F624B7
:1007D000E3240800F624E324E3240800E3240800CB
:1007E000E324E324F624E3240800F624F624E32497
:1007F0000800E324E324E324E3240800E324E324BF
:100800000800E324F624F624F6240800F624E32462
:10081000F6240800E324F624E324E3240800F62465
:10082000F6240800F624E3240800F624F624F6242F
:100830000800E324F624F624E3240800F624F62432
:10084000E324F6240800E324F624E3240800E32448
:10085000E324E3240800F6240800E324E324F62438
:100860000800E324E324E324F6240800E324F62428
:10087000F6240800F624E324E324F6240800F624F2
:10088000E324F624F6240800F624F624E324E324E3
:100890000800F624F624F624F624F6240800E324BF
:1008A000F624F624F624F6240800E324E324F624B0
:1008B000F624F6240800E324E324E324F624F624B3
:1008C0000800E324E324E324E324F6240800E324DB
:1008D000E324E324E324E3240800F624E324E324CC
:1008E000E324E3240800F624F624E324E324E324A9
:1008F0000800F624F624F624E324E3240800F62472
:10090000F624F624F624E3240800E324F624E32462
:10091000F624E324F6240800F624F624E324E32452
:10092000F624F6240800E324E324F624F624E32442
:10093000E3240800F624E324E324F624E324080057
:10094000F624E324E324E324F6240800F624E32435
:10095000E324E324E324F624080086120611400869
:10096000A0004108A1006225080086120611400877
:10097000A0004108A10062254008A0004108A10094
:1009800062254008A0004108A100622508008612E7
:1009900006114008A0004108A10062254008A000FF
:1009A0004108A10062254008A0004108A10062257D
:1009B0004008A0004108A10062254008A0004108AD
:1009C000A100622508008616061506308400403016
:1009D000AA004808A0004908A1004208A200430854
:1009E000A300D52586120611AD240800861606152B
:1009F000063084004030AA004808A0004908A10041
:100A00004408A2004508A300D52586120611AD248E
:100A1000080086160615063084004030AA004808F3
:100A2000A0004908A1004608A2004708A300D52558
:100A300086120611AD240800AF012F080E3C031CDE
:100A4000322D2F08013EAD002D08313E84000008F4
:100A5000AA002F08313E84002A0880000130AF0729
:100A6000031C1D2D1F3083053008C000FE30BF253C
:100A7000C030BF25AF012F080F3C031C482D2F08A5
:100A8000313E84000008A7250130AF07031C3B2D31
:100A90001F30830508004B2D1030A800A101A001D4
:100AA000A70CA60C031C5A2D2208A0072308031824
:100AB000230FA107A10CA00CA50CA40CA80B502D72
:100AC00024080800A00803196D2D7425A003000058
:100AD0000000000000000000622DA10803190800BA
:100AE0007425A103A003622D0C30A500A50B762D63
:100AF000000000001230A200A20B832D8525852561
:100B000000000000080085257C2D0D30A400A40BFA
:100B1000872D000008000A30A802031C0800902D51
:100B20000630A802031C0800902D1030A802000116
:100B3000031C013EA902031C08009E2D0A30A802D6
:100B40000001031C013EA902031C08009E2DA80001
:100B50000516A80EF030850528080F398504BB2539
:100B6000A80EF030850528080F398504BB256430B0
:100B7000A8008B2508008615000086110800A80033
:100B80000512A80EF030850528080F398504BB250D
:100B9000A80EF030850528080F398504BB2588305C
:100BA000A8001330A900952508002A088004200811
:100BB000A8002108A90095250130A202031CA30367
:100BC0002A0980052008A8002108A9009525A20867
:0C0BD000031DD52DA308031DD52D080022
:02400E00503F21
:00000001FF
